:020000040000FA
:040000008A01032846
:0A00060083120313981383160313EB
:1000100007309C009D019B0185018601831203131B
:1000200085018601542027080F394920A30028089C
:100030000F3949200138A40029080F394920A500AB
:10004000FF30A600A201233084003420000886007F
:1000500038203C20840AA20A2208033C031D2628DB
:10006000A603031D22280E288514442085100800AD
:1000700005154420051108002830A000A100A10B9F
:100080003F28A00B3E280800FA30A100A10B46280B
:10009000080082077E340C34B6349E34CC34DA3413
:1000A000F8340E34FE34CE34682083208520EA20D4
:1000B0008520E020682083208520AB208520AD2886
:1000C000B700AD28B6006820EC204F215E21080063
:1000D0006B207E20080083160313851583120313FB
:1000E000831603138511831203138511712183165F
:1000F00003138515831203136821080085197E28D0
:10010000851D80280800CC300800B4000830B500F8
:1001100083160313851583120313831603138511A6
:10012000831203138511B40C031C9C28831603133C
:10013000851583120313A2288316031385118312D6
:10014000031385116B218316031385158312031383
:10015000B50B8D280800BE3008000830AC00AD019A
:100160008316031385158312031383160313851156
:100170008312031385110000831603138515831260
:1001800003136321031085190314AD0C6B2183162F
:100190000313851583120313AC0BB5282D083919E9
:1001A000D528AF003915B9156028B919DE282F02F6
:1001B000031908002D08AF00B9156028B91162288D
:1001C00083160313851583120313851DE5288121EA
:1001D0000000080044300800F22005210F213621DC
:1001E0004A210800BA010330B5000314B60CB70C5D
:1001F000BA0CB50BF5280310B70CBA0C0430B500D7
:100200000310BA0CB50B0029080039100311FF3098
:10021000360503190D293914080039100800031197
:1002200000303A04031932290C303A050319262903
:10023000BA191D293A1D222920293A1924292229CF
:10024000292134292C2134292F2134293130A900A6
:1002500008003330A90008003530A9000800383004
:10026000A9000800B9100800B91408003708BC013B
:10027000BD01BE000A303E02031C4729BE00BD0A74
:100280000A303D02031C3A29BD01BC0A3A293D0E41
:100290003E0708003030BC04BD04BE040800391815
:1002A0005229FA303D08A7003E08A800B91859297C
:1002B0005B29290808003030A90008002E30AA0068
:1002C00008000530732902307329033000007329B8
:1002D0000530000073290F3073291330732916304D
:1002E0007329A6307329B100B10B742908001030AE
:1002F0007929B300FF30B100B10B7C29B30B7A2907
:10030000080001308329B300D930B2001030B100A9
:0E031000B10B8829B20B8629B30B8429080093
:00000001FF
